:020000040000FA
:100000008316FF2390008312850107309900831621
:100010001830850010309500811383120330D20010
:1000200021308500C830432122308500C83043216B
:1000300024308500C8304321D20B10280030B00096
:10004000A101A201A301A401A501A601A701A80184
:10005000A901AA010F30AB001930AC000630AD0089
:10006000AF0124308500A001051A38282E14392844
:100070002E1085194128A00A20087F39031D392830
:100080001C29A001851D4A28A00A2008FF39031D4C
:1000900042281C2985195228A00A2008FF39031D6F
:1000A0004A281C2915302002031C33283030200236
:1000B000031C1C2939302002031CBD28AF1C6428F6
:1000C00045302002031CFF283C302002031C1C2961
:1000D0004A302002031C852858302002031C852842
:1000E0005A302002031C1C2973302002031C85286F
:1000F000AF187C282F1D84288C302002031C1C295B
:10010000A2302002031CE0281C2930181C29A10A57
:100110002E188F282108503C031D382993282108C8
:10012000323C031D3829A101A201A401A501B01B85
:10013000A528A60A2E18A12826082C02031838295B
:10014000A5282608033C031D3829A601A701A901FB
:10015000AA010130AF002E18B4284630AB0006309B
:10016000AD001930AC00BA284630AB000C30AD0001
:100170000330AC00013085003829B0181C29A20AD0
:100180002208723C031D3829A101A201A301A40188
:10019000A501B01BD028A70A27082B02031838296D
:1001A000A601A701A801A901AA010230AF000F30E2
:1001B000AB004630AC001430AD0002308500382969
:1001C000B0181C29A40A2408283C031D3829A101C1
:1001D000A201A301A401A501B01BF328A90A2908C3
:1001E000053C031D3829A601A701A801A901AA0100
:1001F0000430AF000530AB00023085003829B0185C
:100200001C29A30A2308623C031D3829A101A2016D
:10021000A301A401A501B01B1229A80A2808053CC6
:10022000031D3829A601A701A801A901AA010030D0
:10023000AF00243085003829A50A2508643C031D39
:100240003829A101A201A301A401A501B01B2D29F8
:10025000AA0A2A082D0203183829A601A701A80115
:10026000A901AA010630AD000030AF00243085009E
:100270002F1D3328D20AD21F402900308500332891
:10028000023085003328D1003230D0000000000059
:10029000000000000000000000000000D00B462914
:0602A000D10B4429080007
:0207FE000034C5
:02400E00C43FAD
:00000001FF
